:100000000C94F0030C9437040C9437040C943704CC
:100010000C9437040C9437040C9437040C94370474
:100020000C9437040C9437040C94370E0C94090F7D
:100030000C9437040C9437040C9437040C94370454
:100040000C9437040C947D230C9437040C943704DF
:100050000C9437040C940F1D0C9437040C94370443
:100060000C9437040C9437040C9437040C94370424
:100070000C9437040C9437040C9437040C94370414
:100080000C9437040C9437040C9437040C94370404
:100090000C9437040C9437040C9437040C943704F4
:1000A0000C9437040C9437040C943704470451041F
:1000B00069048104C904CF04F004D504EB04E1040D
:1000C000E604DB04B1049904F504760F980F8B1055
:1000D000980F8B10DD0F00108B1055106810521305
:1000E000521381138113C413FE130B160B1617142E
:1000F0000B160C150C15DF150B160B16F61501E17A
:100100000137023702E10138023801E201250225F8
:1001100002E20001E10137023702E1013802380151
:10012000E10130023002E10001E10137023702E172
:100130000138023801E10107020702E1000135023E
:1001400035012002200001E10137023702E10138C8
:10015000023801E10125022502E10001E101360238
:100160003602E10138023801E10125022502E100F1
:1001700001E10136023602E10138023801E10126CF
:10018000022602E10001E10137023702E1013802F3
:100190003801E10126022602E10002E002E201301C
:1001A00002300002E002E20001E001E20002E002AF
:1001B000E3016402640002E002E30001E001E30005
:1001C00002E002E2012E022E02E10002E002E10260
:1001D000E20001E001E101E20002E001E3010602C8
:1001E0000602E30002E00001E00002E001E3011981
:1001F000021902E30002E00001E0000000F0A1F0BB
:10020000A329002B00E200E100358100001E00144C
:100210000004001D710D304D831F001A0016001BD5
:10022000000C304C002000080007000600E1042A02
:10023000002100150009001900E1084A00220017FA
:10024000000A000500000003300130E3000000E276
:1002500000000002540230E7000000E60000000445
:100260005423001C000B00110000002E7F240018F6
:10027000000D00100050004B0025000C000E003651
:100280000052002C00260012000F003700510028F9
:100290000027001300330038714F004E002D002F4F
:1002A000003474E50031810000010001000100010B
:1002B00000010000003A003500310001000100019A
:1002C000003B0035022102350001004C003C001EBD
:1002D0000224062202010001003D002D0224022416
:1002E00004010001003E000100370011040000017C
:1002F000000100010000000100000001000E3001BB
:100300000000000100000001003F00240624022339
:100310000200000100400022042502350001000116
:100320000041002304260235023700010042002468
:100330000425041F021E020100430031002604317F
:1003400002010001004400450001002D02010000EF
:100350000001000100010001000100000001000196
:100360000001000100010001000100F400F200FBA7
:1003700000010001000100F000F100FA000100019D
:10038000000100F500F300FC00010001000100F98C
:1003900000FA00F600000001000100010000000169
:1003A0000000000100A800010000000100000001A1
:1003B0000001000100A900AA0000000100010001E5
:1003C000000100010001000100010001000100AC7A
:1003D000000100B600010001000100AB0050000167
:1003E00000010001000100520051000100AE0001B7
:1003F00000010001004F00000001000100010001A8
:1004000000010000000100010001000100010001E5
:1004100000010001000100010001000100010001D4
:1004200000010001000100010001000100010001C4
:1004300000010001000100010001000100000001B5
:100440000001000100000001000000010004300173
:1004500000000001000000010005300630093001F5
:1004600000000001000A300B3008300100010001DB
:10047000000100073001000100010001000100013E
:100480000001000100010001000100010001000164
:100490000001000100010001000100010001000055
:1004A0000001000100010001000100000001000145
:1004B00000010001000100010001000100500001E5
:1004C0000001000100010052005100010001000183
:1004D00000010001004F00010001000100010001C6
:1004E0000001000100000001000100010000000106
:1004F00000000001000100010000000100000001F7
:10050000003F00520051002302000001004000247F
:100510000021001E00270001004100250022001FCD
:1005200000370001004200260023002000270001C0
:10053000004300300230002402270201004400453D
:1005400000380001000100000001000100E100018D
:1005500000E0000000010001000100010001003D79
:100560000001000100010001000100E000010001A4
:10057000000100010001002C000100010001000148
:100580000001003C00010001000100010000003AF0
:1005900000010001000000010000003B000E3001DE
:1005A0000000000100000001000100010001000145
:1005B0000000000100010001000100010001000134
:1005C0000001000100010001000100010001000123
:1005D0000001000100010001000100010001000113
:1005E0000001000100010001000100010001000004
:1005F0000016034500720067006F0044006F00782A
:1006000000200045005A00000016034500720067F4
:10061000006F0044006F007800200045005A000081
:10062000000403090409026D00040100A0FA090492
:1006300000000103010100092111010001223F0016
:100640000705810308000A090401000103010200F3
:10065000092111010001224D000705820308000A4B
:100660000904020001030000000921110100012218
:1006700036000705830308000A090403000103008C
:10068000000009211101000122390007058403102F
:1006900000011201100100000008EDFE0713010027
:1006A0000102000105010906A101050719E029E77A
:1006B0001500250195087501810205081901290514
:1006C00095057501910295017503910105071900C2
:1006D000297715002501957875018102C00501096A
:1006E00080A101850216010026B7001A01002AB771
:1006F00000751095018100C0050C0901A101850359
:10070000160100269C021A01002A9C027510950110
:100710008100C005010902A1010901A10005091913
:1007200001290515002501950575018102950175C1
:100730000381010501093009311581257F95027575
:1007400008810609381581257F9501750881060500
:100750000C0A38021581257F950175088106C0C0F5
:1007600005010906A101050719E029E71500250182
:100770009508750181029501750881010508190127
:1007800029059505750191029501750391010507EC
:10079000190029FF150025FF950675088100C00086
:1007A00000000000000000000000010204060A0F23
:1007B00017202C3A4A5D71879DB3C7DAE9F5FCFF33
:1007C000FCF5E9DAC7B39D87715D4A3A2C20170F13
:1007D0000A06040201000000000000000000000002
:1007E00011241FBECFEFDAE0DEBFCDBF04B603FE9B
:1007F00027C08091EF019091F001A091F101B0919B
:10080000F2018730904BA740B04BD1F41092EF012A
:100810001092F0011092F1011092F20114BE84B70F
:10082000877F84BF0FB6F894A89580916000886197
:1008300080936000109260000FBEE0E0FFE3099536
:1008400011E0A0E0B1E0ECE9FAE402C005900D92FD
:10085000A433B107D9F721E0A4E3B1E001C01D92B0
:10086000AF3EB207E1F70E947E0B0C944C250C942E
:100870000000462F50E04F30510508F0DEC0FA016D
:10088000EA5AFF4FDC0112968C910C9401258823C3
:1008900021F085EE0E94EC11D0C085EE0E94B412CA
:1008A000CCC0882349F00E94D91C909335018093D5
:1008B000340188EF91E008958091340190913501E1
:1008C0000E94E51C873991050CF0A8C08AEE91E0E2
:1008D0000895882349F00E94D91C90933501809394
:1008E000340187EE91E008958091340190913501B3
:1008F0000E94E51C873991050CF093C089ED91E0C9
:100900000895882349F00E94D91C90933501809363
:10091000340182ED91E00895809134019091350188
:100920000E94E51C873991050CF07EC080EC91E0B7
:100930000895882349F00E94D91C90933501809333
:1009400034018BEB91E00895809134019091350151
:100950000E94E51C873991050CF069C08DEA91E091
:100960000895882349F00E94D91C90933501809303
:10097000340188EA91E00895809134019091350125
:100980000E94E51C873991050CF054C08AE991E07A
:100990000895882309F451C085E891E008958823DB
:1009A00009F44BC080E791E00895882309F445C01D
:1009B0008BE591E00895882309F43FC086E491E037
:1009C00008958823D1F18DE391E008958823A9F15A
:1009D00088E291E00895882381F183E191E0089510
:1009E000882359F18EEF90E00895882331F18091AA
:1009F000B3019091B401A091B501B091B60120E28C
:100A0000822780729927AA27BB278093B3019093EE
:100A1000B401A093B501B093B6010FC085EF91E08A
:100A2000089584EE91E008958BEC91E0089586EBB3
:100A300091E0089583EA91E0089580E090E00895C0
:100A400008956091B3017091B4018091B5019091C6
:100A5000B6010E943C1C56985E9825982D982698C1
:100A60002E9827982F988330C1F028F4813041F0D8
:100A7000823049F00895843049F0853051F008956E
:100A8000259A2D9A0895269A2E9A0895259A2D9A98
:100A900004C0259A2D9A269A2E9A279A2F9A08955D
:100AA0000C94210556985E9825982D9826982E9896
:100AB00027982F988FEF90E090938900809388007B
:100AC00090938B0080938A0090938D0080938C008C
:100AD000259A2D9A2FEF80E792E021508040904098
:100AE000E1F700C00000269A2E9A2FEF80E792E0EF
:100AF000215080409040E1F700C00000279A2F9AD3
:100B00002FEF80E792E0215080409040E1F700C055
:100B1000000025982D982FEF80E792E0215080402B
:100B20009040E1F700C0000026982E982FEF80E754
:100B300092E0215080409040E1F700C000002798EB
:100B40002F9856985E9825982D9826982E98279835
:100B50002F98089589EA8093800089E0809381002E
:100B600024982C983F988AB18F748AB96E98479AC6
:100B70008BB1806B8BB9769A0E9452050C9420053C
:100B800080E2809300018091360181110EC00E94A5
:100B90000F0681E0809336012FEF83ED90E3215023
:100BA00080409040E1F700C0000080E40E941506FC
:100BB0008093000181112EC00E943F0680930001A6
:100BC000811128C00E943F0680930001811122C03C
:100BD0008FE30E943F068093000181111BC00E9499
:100BE000370680E40E94150680930001811112C02F
:100BF0008CE00E943F068093000181110BC00E948F
:100C00003F0680930001811105C08FE30E943F06DB
:100C1000809300010E943706809100010895109290
:100C2000B9008AE08093B800089594EA9093BC00DC
:100C30009091BC0097FFFCCF9091B900987F9830BD
:100C400021F0903111F081E008958093BB0084E899
:100C50008093BC008091BC0087FFFCCF8091B900DD
:100C6000887F883111F0803471F780E0089584E93D
:100C70008093BC008091BC0084FDFCCF08958093DC
:100C8000BB0084E88093BC008091BC0087FFFCCF50
:100C90009091B900987F81E0983209F480E008953E
:100CA00084E88093BC008091BC0087FFFCCF8091DA
:100CB000BB00089580910001811115C080E40E945D
:100CC00015068093000181110CC082E10E943F064D
:100CD00080930001811105C08FEF0E943F06809331
:100CE00000010E94370684B1807F84B985B1807F7E
:100CF00085B98AB1837F8AB98BB1837F8BB93E98DE
:100D0000469808950E94C005809300010E945A06EB
:100D100080B38C7080BB81B3836F81BBE6E4F1E06C
:100D2000A8E3B1E011921D9281E0E435F807D1F714
:100D30000C94AA059F92AF92BF92CF92DF92EF924E
:100D4000FF920F931F93CF93DF938091000188232D
:100D500079F0809137018F5F80933701811108C04E
:100D60000E94C00580930001811102C00E945205BB
:100D700088E3E82E81E0F82E8701C0E0D0E0BB24B4
:100D8000B39492E0A92ECC24C394D12CC730D105C2
:100D900000F580910001811164C080E40E94150675
:100DA00080930001811112C082E10E943F0680936E
:100DB000000181110BC0C6010C2E01C0880F0A94DE
:100DC000EAF780950E943F06809300010E94370653
:100DD00048C0CA30A1F028F4C83059F0C93061F0D9
:100DE00005C0CC3089F070F0CD3089F0209A289879
:100DF00010C0219A29980DC0229A2A980AC0239AD5
:100E00002B9807C0529A01C0539A5B9802C03E9A31
:100E10004698E0EAEA95F1F78FB181708B257999D0
:100E200002C032E001C030E0832B7C9902C034E084
:100E300001C030E0832B7D9902C028E001C020E092
:100E4000822B7E9902C090E101C090E0892B9FB176
:100E50009095991F9927991F9295990F907E892BAC
:100E60000FC08091000181114AC080E40E941506E4
:100E700080930001882381F1912C0E943706892DEF
:100E8000D8019C91981719F08C93A09201010E94AF
:100E90005A0621960F5F1F4FCE30D10509F076CF4D
:100EA00080910101882369F1815080930101882399
:100EB00039F0EFE9FFE03197F1F700C0000021C001
:100EC000E6E4F1E0D7018D917D018193B6E4EB1664
:100ED000B1E0FB06B9F715C083E10E943F0680939D
:100EE00000018111C9CF81E40E94150680930001A1
:100EF0008111C2CF0E945006982E9094BECF80E000
:100F0000BFCF0E94500581E0DF91CF911F910F91DB
:100F1000FF90EF90DF90CF90BF90AF909F9008959B
:100F2000E82FF0E0EA5BFE4F8081089508958B3B47
:100F3000910580F4883A910548F5853A9105D8F4F1
:100F40008430910508F0B2C0019709F06EC081E0CD
:100F500090E00895803E910508F467C0883E9105B1
:100F600008F4A4C09C01205F31092031310508F04C
:100F70005CC090650895853A910509F459C0863A98
:100F8000910509F058C082E890E40895883A9105E7
:100F900009F454C0893A910509F453C08A3A91057D
:100FA00009F452C08B3A910509F451C08C3A91056D
:100FB00009F450C08D3A910509F44FC0803B91056A
:100FC00009F44EC08E3A910509F44DC08F3A91054F
:100FD00009F44CC0813B910509F44BC0823B91055B
:100FE00009F44AC0833B910509F449C0843B91054B
:100FF00009F448C0853B910509F447C0863B91053B
:1010000009F446C0873B910509F445C0883B91052A
:1010100009F444C0893B910509F443C08A3B91051A
:1010200009F442C080E094E4089580E090E00895DF
:1010300081E890E4089583E890E4089582EE94E4D2
:10104000089589EE94E408958AEE94E4089585EB7A
:1010500094E4089586EB94E4089587EB94E408956E
:101060008CEC94E408958DEC94E4089583E895E481
:1010700008958AE895E4089582E995E4089584E95D
:1010800095E4089581E296E4089583E296E4089554
:1010900084E296E4089585E296E4089586E296E473
:1010A000089587E296E408958AE296E40895089503
:1010B00024E5829FC0011124FC0126E0729FE00D0F
:1010C000F11D1124E60FF11DEE0FFF1FEF5FFD4F25
:1010D000859194910895880F991FFC01E558FF4F61
:1010E000859194910895880F991FFC01E550FE4F5A
:1010F00085919491089524E5829FC0011124FC01FB
:1011000046E0749FE00DF11D1124E60FF11DEE0F76
:10111000FF1FEF5FFD4F859194919C013A9521153A
:101120004FE1340708F425C13F512115304120F427
:101130009F700E94730808959C013053211530411F
:1011400018F49927906C0895811520E5920769F4A9
:101150000E942D164FEF84E39CE041508040904068
:10116000E1F700C000000C94341D813020E59207A7
:1011700031F48091CE0181608093CE0108959C016D
:1011800030552115304108F05CC0292F33272F70CE
:10119000332721303105E9F4AC0164E0440F551FD9
:1011A0006A95E1F744275370BC016370772702C04A
:1011B000220F331F6A95E2F73C68242B352B73E02E
:1011C000880F991F7A95E1F780769927822B932BC8
:1011D00008952230310529F4982F8827816F906A6D
:1011E000089523303105A1F4AC0133E0440F551FBD
:1011F0003A95E1F7407E57708370992721E030E0FF
:1012000002C0220F331F8A95E2F7C9019C6816C0FD
:101210002430310531F5AC0123E0440F551F2A95E8
:10122000E1F7407E57708370992721E030E002C0DB
:10123000220F331F8A95E2F7C9019A68842B952BF8
:1012400008959C0130572115304118F49F70906229
:1012500008959C0130582115304118F49F70906A10
:101260000895803E9105E0F4803C910558F5813366
:10127000910509F46FC048F48932910509F463C0FF
:101280008A32910509F46DC072C089339105E9F085
:1012900082389105D1F08533910509F44DC067C0BE
:1012A000833E910581F138F4803E9105B9F0823E8C
:1012B0009105D9F05CC0863E910561F1873E9105AC
:1012C000A1F155C00E946B0808952091E00120FD16
:1012D00002C021FF4CC080EE90E049C08091E00147
:1012E00080FFF9CF89E390E042C08091E00182FF66
:1012F0000EC08091E00184FF03C080E090E037C021
:1013000083EE90E034C08091E00182FFF2CF82EE64
:1013100090E02DC08091E00183FF0BC08091E0013F
:1013200084FDEBCF87EE90E022C08091E00183FF47
:10133000F5CF86EE90E01BC08091E00185FF07C0ED
:1013400089E290E014C08091E00185FFF9CF85E348
:1013500090E00DC08091E00186FF07C08AE290E036
:1013600006C08091E00186FFF9CF81E390E00E9402
:10137000970708950895809164010895CF93DF93AE
:1013800000D01F92CDB7DEB79C018091E60184307A
:1013900019F593E099833B832A839093E9008FEFBB
:1013A0009091E800815095FD06C095ED9A95F1F772
:1013B00000008111F5CF8091E80085FF0DC040E06D
:1013C00050E063E070E0CE0101960E942B0C80910A
:1013D000E8008E778093E8000F900F900F90DF91D8
:1013E000CF910895CF93DF9300D01F92CDB7DEB792
:1013F0002091E601243021F522E029839B838A8312
:1014000083E08093E9008FEF9091E800815095FD93
:1014100006C095ED9A95F1F700008111F5CF809106
:10142000E80085FF0DC040E050E063E070E0CE01D1
:1014300001960E942B0C8091E8008E778093E80043
:101440000F900F900F90DF91CF9108959C018091A4
:10145000E6018430F9F482E08093E9009FEF809107
:10146000E800915085FD06C085ED8A95F1F70000F2
:101470009111F5CF8091E80085FF0CC040E050E06D
:1014800065E070E0C9010E942B0C8091E8008E7726
:101490008093E8000895CF93DF93EC018091E601FB
:1014A000843009F046C090910C019923D9F09091B5
:1014B0000D019923B9F08093E9008FEF9091E80036
:1014C000815095FD06C095E19A95F1F700008111D4
:1014D000F5CF8091E80085FF2CC040E050E060E14E
:1014E00070E017C081E08093E9008FEF9091E800F1
:1014F000815095FD06C095ED9A95F1F70000811198
:10150000F5CF8091E80085FF14C040E050E068E02E
:1015100070E0CE010E942B0C8091E8008E778093C2
:10152000E80080E1FE01A4E5B1E001900D928A950A
:10153000E1F7DF91CF9108958091E501811109C014
:101540000E94BC0D0E94190E8091E200846080937D
:10155000E20008951092E501089508950C946A231D
:101560000E94CA1C0E9470230E94C4100C94BA09E5
:1015700042E061EC81E00E94350D42E061EC82E0E6
:101580000E94350D42E061EC83E00E94350D42E19E
:1015900061EC84E00C94350D8091E801833009F40E
:1015A00055C030F4813071F0823009F48EC0089556
:1015B0008A3009F47AC08B3009F460C0893009F0B0
:1015C0009CC020C08091E701813A09F096C08091CB
:1015D000E800877F8093E8008091EB019091EC0117
:1015E000892B21F460E184E591E003C060E080E0B4
:1015F00090E070E00E94760C8091E8008B778093F9
:10160000E80008958091E701813209F076C0809169
:10161000EB019091EC01009719F0039709F06DC070
:101620008091E800877F8093E8008091E80082FD48
:1016300005C08091E6018111F8CF5FC08091F10073
:10164000809364018091E8008B7753C08091E7011B
:10165000813A09F052C08091EB019091EC01892B05
:1016600009F04BC08091E800877F8093E80080916B
:10167000E80080FFFCCF80910C0136C08091E7012B
:101680008132D9F58091EB019091EC01892BA9F57C
:101690008091E800877F8093E8000E946A0D809126
:1016A000E90180930C010C942D168091E7018132A1
:1016B00021F58091E800877F8093E8000E946A0D01
:1016C0008091EA018093650108958091E701813A54
:1016D000A1F48091E800877F8093E8008091E80082
:1016E00080FFFCCF809165018093F1008091E8003C
:1016F0008E778093E8000C946A0D089584B7877FF5
:1017000084BF0FB6F894A89580916000886180939B
:101710006000109260000FBE90E080E80FB6F89471
:1017200080936100909361000FBE0E9413110E948C
:10173000BC0D0E94190E8091E20084608093E2004B
:1017400078940E94A4100E94151182E091E00E94FA
:10175000BF100E9458238091E601853069F40E94F1
:101760008C1C8091E4018823B1F30E94B61C88236D
:1017700091F30E94150CEFCF0E941B11ECCF292F83
:10178000332723303105C9F060F42130310581F071
:101790002230310509F041C08DE690E025E236E0C7
:1017A00040C021323105E1F02232310531F135C03E
:1017B00082E190E022E936E034C09927813091053A
:1017C00049F028F0029749F5E1EFF5E005C0E1E2C4
:1017D000F6E002C0E9E0F6E0849190E09F0121C0CC
:1017E0006430D8F4E62FF0E0EE0FFF1FEE5DFE4F01
:1017F0002081318189E090E014C0643070F470E0A1
:10180000FB01EE0FFF1FE65EFE4F20813181FB01E1
:10181000EA5EFE4F808190E004C080E090E020E02E
:1018200030E0FA0131832083089580E189BD82E1AF
:1018300089BD09B400FEFDCF8091D8008F7D8093D3
:10184000D8008091E00082608093E0008091E00009
:1018500081FDFCCF0895CF92DF92EF92FF920F931C
:101860001F93CF93DF93EC018B016A010E94890DD6
:10187000811133C0C114D10439F0F6018081918106
:10188000081B190BC80FD91FE12CF12C01151105EC
:1018900019F18091E80085FD16C08091E8008E77EF
:1018A0008093E800C114D10449F0F6018081918150
:1018B000E80EF91EF182E08285E00FC00E94890DDA
:1018C000882321F30AC089918093F1000150110906
:1018D000FFEFEF1AFF0ADACF80E0DF91CF911F917F
:1018E0000F91FF90EF90DF90CF9008952091ED0140
:1018F0003091EE012617370748F06115710539F46C
:101900002091E8002E772093E80001C0B901FC0186
:1019100020E06115710579F18091E6018823F1F1EC
:101920008530F1F18091E80083FD3CC08091E800B2
:1019300082FD2EC08091E80080FFEBCF2091F30064
:101940008091F20090E0922B6115710551F0883082
:10195000910538F421912093F100615071090196AD
:10196000F3CF21E0089709F020E08091E8008E771E
:101970008093E800CECF2111CFCF0AC08091E6013D
:10198000882361F0853061F08091E80083FD0AC012
:101990008091E80082FFF2CF80E0089582E0089510
:1019A00083E0089581E008952091ED013091EE01EA
:1019B0002617370748F06115710539F42091E800C2
:1019C0002E772093E80001C0B901FC0120E06115E9
:1019D000710591F18091E601882309F440C08530BA
:1019E00009F43FC08091E80083FD3DC08091E8008C
:1019F00082FD2FC08091E80080FFE9CF2091F300A5
:101A00008091F20090E0922B6115710559F08830B9
:101A1000910540F424912093F100319661507109B1
:101A20000196F2CF21E0089709F020E08091E800CC
:101A30008E778093E800CBCF2111CCCF0AC0809164
:101A4000E601882361F0853061F08091E80083FD34
:101A50000AC08091E80082FFF2CF80E0089582E022
:101A6000089583E0089581E00895982F973068F5F0
:101A70009093E900981739F07091EC002091ED00F7
:101A80005091F00003C0242F762F50E021FD02C0BA
:101A90009F5FECCF3091EB003E7F3093EB003091B5
:101AA000ED003D7F3093ED003091EB0031603093DD
:101AB000EB007093EC002093ED005093F000209128
:101AC000EE0027FDE5CF80E008958F708093E90058
:101AD00081E008958091E70187FF11C08091E800BF
:101AE00082FD05C08091E6018111F8CF11C080917F
:101AF000E8008B770BC08091E601882349F0809144
:101B0000E80080FFF8CF8091E8008E778093E800AE
:101B100008952091E4003091E50095E64091EC00B5
:101B2000842F817040FF23C08091E80080FD1DC09C
:101B30008091E601882399F0853099F08091EB003F
:101B400085FD11C04091E4005091E5002417350750
:101B500029F3915011F09A01E1CF84E0089582E0D9
:101B6000089583E0089581E0089580E0089540910C
:101B7000E80042FFDDCF08950E942A0E0E94320E37
:101B8000E0EEF0E0808181608083E8EDF0E080812C
:101B90008F77808319BCA7EDB0E08C918E7F8C93FA
:101BA00080818F7E80831092E50108950F931F93AB
:101BB000CF93DF930E942A0E0E94320EC8EDD0E030
:101BC00088818F77888388818068888388818F7DEA
:101BD000888319BC1092E6011092E2011092E40190
:101BE0001092E30100EE10E0F80180818B7F80838A
:101BF00088818160888342E060E080E00E94350D4A
:101C0000E1EEF0E080818E7F8083E2EEF0E0808183
:101C100081608083808188608083F80180818E7FED
:101C20008083888180618883DF91CF911F910F919C
:101C30000895E8EDF0E080818F7E8083E7EDF0E0AD
:101C400080818160808384E082BF81E08093E501B0
:101C50000C94D60DE8EDF0E080818E7F80831092A9
:101C6000E20008951092DA001092E10008951F92A8
:101C70000F920FB60F9211242F933F934F935F93C0
:101C80006F937F938F939F93AF93BF93EF93FF9344
:101C90008091E10082FF0BC08091E20082FF07C0CB
:101CA0008091E1008B7F8093E1000E94A3108091DE
:101CB000DA0080FF1FC08091D80080FF1BC0809198
:101CC000DA008E7F8093DA008091D90080FF0DC00A
:101CD00080E189BD82E189BD09B400FEFDCF81E0CC
:101CE0008093E6010E949C0A05C019BC1092E6018F
:101CF0000E94AA0A8091E10080FF19C08091E20051
:101D000080FF15C08091E2008E7F8093E200809179
:101D1000E20080618093E2008091D800806280932D
:101D2000D80019BC85E08093E6010E94AE0A80913C
:101D3000E10084FF30C08091E20084FF2CC080E18C
:101D400089BD82E189BD09B400FEFDCF8091D80034
:101D50008F7D8093D8008091E1008F7E8093E10099
:101D60008091E2008F7E8093E2008091E2008160AA
:101D70008093E2008091E201882311F084E007C0A3
:101D80008091E30087FD02C081E001C083E0809381
:101D9000E6010E94B00A8091E10083FF29C0809192
:101DA000E20083FF25C08091E100877F8093E100FE
:101DB00082E08093E6011092E2018091E1008E7F43
:101DC0008093E1008091E2008E7F8093E200809119
:101DD000E20080618093E20042E060E080E00E94E7
:101DE000350D8091F00088608093F0000E94AD0A6C
:101DF000FF91EF91BF91AF919F918F917F916F91E3
:101E00005F914F913F912F910F900FBE0F901F90B8
:101E100018951F920F920FB60F9211242F933F9394
:101E20004F935F936F937F938F939F93AF93BF93E2
:101E3000CF93DF93EF93FF93C091E900CF70809130
:101E4000EC00D82FD17080FDD0E81092E90080918D
:101E5000F000877F8093F00078940E944D0F1092DD
:101E6000E9008091F00088608093F000CD2BCF7066
:101E7000C093E900FF91EF91DF91CF91BF91AF91B6
:101E80009F918F917F916F915F914F913F912F9192
:101E90000F900FBE0F901F9018951F93CF93DF9355
:101EA000CDB7DEB7AA970FB6F894DEBF0FBECDBF91
:101EB000E7EEF1E08091F100819321E0EF3EF2073F
:101EC000C9F70E94CC0A8091E80083FF24C1809169
:101ED000E7019091E801492F50E04A30510508F0A0
:101EE0001AC1FA01EB59FF4F0C940125803881F09B
:101EF000823809F010C18091EB018F708093E90066
:101F00008091EB0085FB882780F91092E90006C0DC
:101F10008091E3019091E401911182609091E80039
:101F2000977F9093E8008093F1001092F100C8C071
:101F3000282F2D7F09F0EFC0882319F0823061F03F
:101F4000EAC08091E901813009F0E5C0933009F0E1
:101F500080E08093E4012BC08091E901811127C0CA
:101F60008091EB018F7009F4D6C08093E900209135
:101F7000EB0020FF1CC0933021F48091EB008062C5
:101F800014C09091EB0090619093EB0021E030E061
:101F9000A90102C0440F551F8A95E2F74093EA0059
:101FA0001092EA008091EB0088608093EB00109221
:101FB000E9008091E800877F86C08111ACC0109154
:101FC000E9011F778091E3008078812B8093E30003
:101FD0008091E800877F8093E8000E946A0D8091DD
:101FE000E80080FFFCCF8091E30080688093E300ED
:101FF000111102C082E001C083E08093E6018BC032
:102000008058823008F087C08091E9019091EA0100
:102010008C3D53E0950779F583E08A838AE28983D2
:102020004FB7F894DE01139620E03EE051E2E32F33
:10203000F0E050935700E49120FF03C0E295EF7069
:102040003F5FEF708E2F90E0EA3010F0C79601C02E
:10205000C0968D939D932F5F243149F74FBF809198
:10206000E800877F8093E8006AE270E0CE01019685
:102070000E94760C14C0AE014F5F5F4F6091EB0180
:102080000E94BF0BBC01892B09F445C09091E80068
:10209000977F9093E80089819A810E94D40C809167
:1020A000E8008B778093E80036C08038A1F58091F6
:1020B000E800877F8093E8008091E2018093F1003F
:1020C0008091E8008E778093E8000E946A0D23C01B
:1020D000811121C08091E9019091EA01992702972D
:1020E000D4F48091E800877F8093E8008091E90133
:1020F0008093E2010E946A0D8091E201811106C085
:102100008091E30087FD02C081E001C084E08093FC
:10211000E6010E94B80A8091E80083FF0AC080911E
:10212000E800877F8093E8008091EB0080628093D5
:10213000EB00AA960FB6F894DEBF0FBECDBFDF91BD
:10214000CF911F9108950895CF938091E601882340
:10215000A1F0C091E900CF709091EC00892F8170BF
:1021600090FD80E8C82B1092E9008091E80083FD83
:102170000E944D0FCF70C093E900CF9108959093C6
:102180006B0180936A010895E0916A01F0916B01FF
:10219000309721F00190F081E02D099480E00895BE
:1021A000E0916A01F0916B01309721F00280F38198
:1021B000E02D09940895E0916A01F0916B01309748
:1021C00021F00480F581E02D0994089520916801A3
:1021D000309169012817390771F090936901809354
:1021E0006801E0916A01F0916B01309721F006805F
:1021F000F781E02D099408952091660130916701DF
:102200002817390771F09093670180936601E09178
:102210006A01F0916B01309721F00084F185E02D87
:102220000994089508950C9412110E94D01C0E94E4
:1022300082060C94961DCF92DF92EF92FF920F933D
:102240001F93CF93DF93CDB7DEB72B970FB6F894DC
:10225000DEBF0FBECDBF0E949A068DE6C82E81E07C
:10226000D82E00E010E0E02E802F0E949007F601AB
:1022700041916F01F82EF426B1F40F5F1F4F0E301D
:10228000110589F78FEF89838A831B820E94D91CED
:102290008160782F9D838C8349815A816B818D81E8
:1022A0000E94BE1140C09091CE0191FF04C08B8767
:1022B0000E9496078B8520E030E04F2D50E0922F52
:1022C000BA01022E02C0759567950A94E2F760FF85
:1022D00024C02E83EF8221E030E0690102C0CC0CE3
:1022E000DD1C9A95E2F790E08C219D21892B09F461
:1022F00020E028870E94D91C8160782F9A878987DF
:102300004E815F8168858A850E94BE11F801E3597C
:10231000FE4F8081C826C08206C02F5F3F4F263007
:10232000310569F6AACF0E947D200E94C4109091C9
:102330006C018917A1F00E94C41080936C012B9648
:102340000FB6F894DEBF0FBECDBFDF91CF911F91C6
:102350000F91FF90EF90DF90CF900C94BA092B96DD
:102360000FB6F894DEBF0FBECDBFDF91CF911F91A6
:102370000F91FF90EF90DF90CF900895CF93DF9370
:10238000CDB7DEB72B970FB6F894DEBF0FBECDBF2B
:102390004F83588769877A878B87DE01119686E09D
:1023A000FD0111928A95E9F785E0FE0137960190CB
:1023B0000D928A95E1F749815A816B817C818D81EB
:1023C0009E810E94C1182B960FB6F894DEBF0FBEF7
:1023D000CDBFDF91CF910895CF93C82F882309F403
:1023E000C1C0823859F40E94C41081FDBBC089E38A
:1023F0000E945E1B0E94161C89E30CC0833879F48E
:102400000E94C41080FDAEC083E50E945E1B0E9446
:10241000161C83E50E949D1BCF910C94161C8438DA
:1024200059F40E94C41082FD9DC087E40E945E1B87
:102430000E94161C87E4EECF8CEF8C0F813A48F493
:102440008C2F0E94BD2281118DC08C2F0E945E1B9B
:10245000E3CF80E28C0F883048F4C77081E001C080
:10246000880FCA95EAF70E94DF1BD6CF8BE58C0F49
:10247000833078F4C53A29F0C63A31F083E890E029
:1024800005C081E890E002C082E890E0CF910C9412
:10249000E61088E58C0F833108F064C0C83A39F142
:1024A000C93A41F1CA3A49F1CB3A51F1CC3A59F122
:1024B000CD3A61F1C03B69F1CE3A71F1CF3A79F191
:1024C000C13B81F1C23B89F1C33B91F1C43B99F11E
:1024D000C53BA1F1C63BA9F1C73BB1F1C83BB9F17E
:1024E000C93BC1F1CA3BC9F180E090E038C082EE3F
:1024F00090E035C089EE90E032C08AEE90E02FC0C7
:1025000085EB90E02CC086EB90E029C087EB90E053
:1025100026C08CEC90E023C08DEC90E020C083E8D6
:1025200091E01DC08AE891E01AC082E991E017C0ED
:1025300084E991E014C081E292E011C083E292E06C
:102540000EC084E292E00BC085E292E008C086E211
:1025500092E005C087E292E002C08AE292E0CF9169
:102560000C94FC10CF910895882309F44BC0823855
:1025700059F40E94C41081FF45C089E30E945E1B8C
:102580000E94161C89E30CC0833871F40E94C410A9
:1025900080FF38C083E50E945E1B0E94161C83E505
:1025A0000E949D1B0C94161C843859F40E94C41080
:1025B00082FF28C087E40E945E1B0E94161C87E4ED
:1025C000EFCF9CEF980F913A58F390E2980F983024
:1025D00050F4877091E001C0990F8A95EAF7892F2E
:1025E0000E94E51BDFCF9BE5980F933020F480E03D
:1025F00090E00C94E610885A833120F480E090E05B
:102600000C94FC100895882321F00E94DF1B0C9489
:10261000161C0895882321F00E94E51B0C94161CBB
:102620000895BF92CF92DF92EF92FF920F931F9384
:10263000CF93DF9300D000D000D0CDB7DEB77C01C0
:1026400085E0F701DE01119601900D928A95E1F780
:10265000F70183819481892B09F4DDC29081818106
:102660008F3F19F49F3F09F4D6C2F70102812581FB
:1026700022952F7099838A8389819A812E830E9463
:102680001D1B182FB92E0E941C1B0E94E319EB2D55
:10269000E295EF704E2F50E0FA01E159FF4F2E8185
:1026A0000C9401258B2D807F9B2D9F70F92E882304
:1026B00019F0F29480EFF822002349F0FF2009F48A
:1026C00057C28F2D0E94EF1B0E94161C51C2812FF2
:1026D0000E94B412FF2009F49EC28F2D0E94F51BA8
:1026E00026960FB6F894DEBF0FBECDBFDF91CF9117
:1026F0001F910F91FF90EF90DF90CF90BF900C94BF
:10270000161C3B2D307F8B2D8F70303211F082954F
:10271000807F112319F0113021F12CC00023B9F072
:10272000222309F490C1213009F08DC126960FB6FD
:10273000F894DEBF0FBECDBFDF91CF911F910F91F7
:10274000FF90EF90DF90CF90BF900C94FF1B22235F
:1027500019F0213009F45FC28E830E94021C8E8121
:1027600086C1002321F0223008F055C26CC121112E
:1027700052C27DC1002321F0222309F464C1F8C1B3
:10278000222309F474C109C28B2D86958695837026
:1027900019F08130D1F03FC2002321F0812F9B2D11
:1027A000937002C080E090E026960FB6F894DEBFEA
:1027B0000FBECDBFDF91CF911F910F91FF90EF9092
:1027C000DF90CF90BF900C94E610002321F0812F72
:1027D0009B2D937002C080E090E026960FB6F8948F
:1027E000DEBF0FBECDBFDF91CF911F910F91FF9044
:1027F000EF90DF90CF90BF900C94FC10812F0023BE
:1028000019F00E94851F02C00E94ED1F26960FB688
:10281000F894DEBF0FBECDBFDF91CF911F910F9116
:10282000FF90EF90DF90CF90BF900C9472208B2D93
:10283000837009F075C00111EEC1812F82958695D4
:102840008770880F880F912F9F70C92ED12CE12C93
:10285000F12C082E04C0CC0CDD1CEE1CFF1C0A94CD
:10286000D2F714FF12C00FE010E020E030E004C007
:10287000000F111F221F331F8A95D2F7C901B8011B
:10288000609570958095909503C060E070E0CB01F5
:102890004B2D4695469543704230C1F060F56C294A
:1028A0007D298E299F29413051F126960FB6F89443
:1028B000DEBF0FBECDBFDF91CF911F910F91FF9073
:1028C000EF90DF90CF90BF900C940A1A6C297D296D
:1028D0008E299F2926960FB6F894DEBF0FBECDBF76
:1028E000DF91CF911F910F91FF90EF90DF90CF90EC
:1028F000BF900C94261A0E940A1AC701B6012696A8
:102900000FB6F894DEBF0FBECDBFDF91CF911F9100
:102910000F91FF90EF90DF90CF90BF900C94EE1945
:10292000002319F08B2D817001C08695882309F44E
:1029300072C1812F829586958770880F880F912F9D
:102940009F70C92ED12CE12CF12C082E04C0CC0C88
:10295000DD1CEE1CFF1C0A94D2F714FF12C00FE01E
:1029600010E020E030E004C0000F111F221F331FD1
:102970008A95D2F7C901B8016095709580959095B8
:1029800003C060E070E0CB014B2D46954695437047
:102990004230C1F060F56C297D298E299F29413094
:1029A00051F126960FB6F894DEBF0FBECDBFDF9172
:1029B000CF911F910F91FF90EF90DF90CF90BF903C
:1029C0000C94E41A6C297D298E299F2926960FB62E
:1029D000F894DEBF0FBECDBFDF91CF911F910F9155
:1029E000FF90EF90DF90CF90BF900C94001B0E945F
:1029F000E41AC701B60126960FB6F894DEBF0FBEE3
:102A0000CDBFDF91CF911F910F91FF90EF90DF909D
:102A1000CF90BF900C94C81A103FD1F118F4103E1B
:102A200050F4A1C0123F09F463C008F44CC0133F36
:102A300009F473C098C01F708B2D8F710023A1F013
:102A40000E94611A812F26960FB6F894DEBF0FBE42
:102A5000CDBFDF91CF911F910F91FF90EF90DF904D
:102A6000CF90BF900C9403130E94821A812F269658
:102A70000FB6F894DEBF0FBECDBFDF91CF911F918F
:102A80000F91FF90EF90DF90CF90BF900C940A13BE
:102A90000023A9F02111BFC08B2D8F7126960FB690
:102AA000F894DEBF0FBECDBFDF91CF911F910F9184
:102AB000FF90EF90DF90CF90BF900C94A71A223038
:102AC00008F0A9C0E9CF0023A9F08B2D8F712696BD
:102AD0000FB6F894DEBF0FBECDBFDF91CF911F912F
:102AE0000F91FF90EF90DF90CF90BF900C94611A00
:102AF000002359F38B2D8F7126960FB6F894DEBF05
:102B00000FBECDBFDF91CF911F910F91FF90EF903E
:102B1000DF90CF90BF900C94821A002399F08B2DF8
:102B20008F7126960FB6F894DEBF0FBECDBFDF9132
:102B3000CF911F910F91FF90EF90DF90CF90BF90BA
:102B40000C944C1A26960FB6F894DEBF0FBECDBF7C
:102B5000DF91CF911F910F91FF90EF90DF90CF9079
:102B6000BF900C94421A0023A9F0222309F4ADCFA0
:102B7000812F26960FB6F894DEBF0FBECDBFDF9132
:102B8000CF911F910F91FF90EF90DF90CF90BF906A
:102B90000C94EC11222309F4ADCF812F26960FB6A9
:102BA000F894DEBF0FBECDBFDF91CF911F910F9183
:102BB000FF90EF90DF90CF90BF900C94B4124B2D0C
:102BC0004F70612FC7010E94390426960FB6F89402
:102BD000DEBF0FBECDBFDF91CF911F910F91FF9050
:102BE000EF90DF90CF90BF900C9466194B2D4F70F3
:102BF000612FC70126960FB6F894DEBF0FBECDBF7A
:102C0000DF91CF911F910F91FF90EF90DF90CF90C8
:102C1000BF900C94570826960FB6F894DEBF0FBEEF
:102C2000CDBFDF91CF911F910F91FF90EF90DF907B
:102C3000CF90BF9008950E94FC1B0E94D11B0E9460
:102C4000161C0E9422210E94722080E090E00E94C7
:102C5000E61080E090E00C94FC100E94EC1B0C94B9
:102C60001B160E941D1B292F22952F702C3030F42B
:102C70002A3048F42250223078F405C02C3041F03C
:102C80002F3031F009C0803E48F0803F29F406C063
:102C900093FB882780F9089580E0089581E00895E6
:102CA000CF93DF9300D000D01F92CDB7DEB70F9047
:102CB0000F900F900F900F90DF91CF910895CF93C9
:102CC000DF9300D000D000D0CDB7DEB726960FB688
:102CD000F894DEBF0FBECDBFDF91CF9108951F9353
:102CE000CF93DF93C0917B0116E080917C01C817E0
:102CF00099F0D0E01C9FF0011D9FF00D1124E358C6
:102D0000FE4F4081518162817381848195810E944F
:102D10005F162196C770E9CFDF91CF911F9108957B
:102D20004091AD015091AE016091AF017091B00141
:102D30008091B1019091B2010C945F168091B20123
:102D400082958F7009F054C08091AF01882309F4F7
:102D50004FC080917B01A0917C014091B0015091C6
:102D6000B1016091AD017091AE01B6E08A1709F42E
:102D70003FC090E041155105C1F17F3F11F46F3F15
:102D8000A1F1B89FF001B99FF00D1124E358FE4F57
:102D9000218127132AC02081261327C022812111D7
:102DA00024C0238134812417350710F421503109C0
:102DB000241B350B283C3105C0F42091B2012F7043
:102DC00020612093B20126E0289FF001299FF00D99
:102DD0001124EE57FE4F80818F70806180838DEAD1
:102DE00091E00E9411130C946F1601968770BECF6C
:102DF0000895CF92DF92EF92FF920F931F93CF939C
:102E0000DF93CDB7DEB762970FB6F894DEBF0FBE83
:102E1000CDBF8C0185E0F801DE011D9601900D9279
:102E20008A95E1F7D8014C9111965C911197129611
:102E30006C918091B0019091B101009709F475C136
:102E40003091AD017091AE017F3F19F43F3F09F41D
:102E50006CC1F801C380D480E090AF01EE2009F48A
:102E6000BEC02091B201C816D90628F0D601A81B11
:102E7000B90BCD0104C0809590958C0D9D1DFF244C
:102E8000F394883C910578F0F12C207F09F0C4C0C0
:102E90007C2DD98AC88A89890E9450168DEA91E0D2
:102EA0000E941113AFC0822F807F09F045C05713D5
:102EB00013C0431311C061110FC02F702061209304
:102EC000B2010E9490168DEA91E00E941113809148
:102ED000B201F80185832EC0CD2819F15F3F11F4AE
:102EE0004F3FF9F0F62E61111CC080917B012091BB
:102EF0007C0136E0821709F45BC090E0389FF00156
:102F0000399FF00D1124E358FE4F7181571306C00D
:102F10007081471303C07281711103C001968770DD
:102F2000E9CFF62E662309F41CC18091B2018160BD
:102F30008093B201F12C15C1571309C0431307C088
:102F4000611105C08091B201F8018583C8C04D8729
:102F50005E878D859E856A8B0E9431166A898823DB
:102F6000D1F16623C1F12091B201822F82958F7039
:102F700090E0029774F08091AD019091AE01988736
:102F80008F831986DB86CA862C87CE0107960E941E
:102F9000111386E0F801ADEAB1E001900D928A9537
:102FA000E1F70E949E160E949016FF24F394D9C068
:102FB0004D875E878D859E850E941D1B292F22953A
:102FC0002F70223008F0C1C09F7009F0BBC0805E36
:102FD000883008F4C6C0C8010E941113E6CFC81695
:102FE000D90608F453C0F601E81BF90BCF01883C61
:102FF000910508F450C0F12C7C2DD98AC88A8989A2
:103000000E945016EDEAF1E086E0DF011D928A95FC
:10301000E9F70E949016A5C0571314C0431312C0BD
:10302000611110C08091B201F8018583C8010E942E
:10303000111386E0EDEAF1E0DF011D928A95E9F7D0
:10304000FE2C8FC04D875E878D859E856A8B0E9482
:1030500031166A89882309F4BECF662309F4BBCFF1
:103060002091B201822F82958F7090E002970CF42C
:1030700090CF8091AD019091AE019A8389831B829C
:10308000DD82CC822E83CE01019681CF80959095F2
:103090008C0D9D1DACCFF62E662309F49CCF5713E3
:1030A00033C0431331C02091B20120FD24C0822FD0
:1030B00082958F70482F50E041155105E1F0D801FD
:1030C00015962C9315974F30510549F08F5F982F27
:1030D0009295907F822F8F70892B15968C93C801C3
:1030E0000E94111386E0F801ADEAB1E001900D9263
:1030F0008A95E1F78ECF86E0F801ADEAB1E0019064
:103100000D928A95E1F72DC04D875E878D859E854E
:103110000E94311681113DCF8091B2018160809370
:10312000B201C8010E9411131CC0662309F453CFD9
:103130004D875E878D859E850E943116882309F410
:103140004ACF27CF811143CF0CC0243008F043CFA2
:103150009F7009F43CCFD80115969C91907F09F09F
:1031600036CF8F2D62960FB6F894DEBF0FBECDBF5F
:10317000DF91CF911F910F91FF90EF90DF90CF9053
:1031800008951F93CF93DF93CDB7DEB72C970FB67B
:10319000F894DEBF0FBECDBF4F83588769877A870B
:1031A0008B879C87CE0107960E94F916882371F0C1
:1031B0008A859B85892B09F441C088858F3F09F05A
:1031C00065C08F818F3F09F061C038C086E0FE0185
:1031D0003796DE01119601900D928A95E1F76A8586
:1031E0007B856115710551F1FF81E885EF3F11F491
:1031F000FF3F21F120917C0130E0C90101968770E9
:10320000992740917B0150E08417950709F447C046
:10321000F983EA837D836C8396E0929FD001939F2C
:10322000B00D1124A358BE4FFE01319601900D92AE
:103230009A95E1F780937C010E946F1616E08091C9
:103240007B0190917C018917B9F1189FC00111246D
:1032500083589E4F0E94F916882371F1E0917B01FB
:103260001E9FF0011124E358FE4F4081518162817D
:103270007381848195810E945F1680917B0190E02B
:1032800001968770992780937B01D9CF4F8158850C
:1032900069857A858B859C850E945F16CFCF0E94B9
:1032A0002D1610927C0110927B01EDEAF1E086E090
:1032B000DF011D928A95E9F72C960FB6F894DEBFD0
:1032C0000FBECDBFDF91CF911F910895EF92FF9276
:1032D0000F931F93CF93DF938C01892B09F46CC05C
:1032E000F12CEE24E394E8012196F80184918437CF
:1032F00040F4843008F051C0813081F0823019F1FF
:103300005BC0853709F444C0A8F19CE7980F90375B
:1033100008F052C08F770E94B41241C00E5F1F4F59
:10332000FE01849190E2980F983050F48770FE2D42
:1033300001C0FF0F8A95EAF78F2F0E94EF1B14C080
:103340000E94EC112DC00E5F1F4FFE01849190E290
:10335000980F983060F48770FE2D01C0FF0F8A959A
:10336000EAF78F2F0E94F51B0E94161C19C00E94BD
:10337000B41216C00E5F1F4FFE01C491CC2381F022
:103380008FE99FE00197F1F700C00000C150F6CF30
:103390000E5F1F4FFE01F49003C00E94EC118E01DE
:1033A0008F2D882309F49FCFEFE9FFE03197F1F7E4
:1033B00000C000008150F5CFDF91CF911F910F9198
:1033C000FF90EF90089508956093B7017093B8014E
:1033D0008093B9019093BA010C941B160F931F931D
:1033E0000091B7011091B8012091B9013091BA0153
:1033F000DC01CB01802B912BA22BB32B8093B70147
:103400009093B801A093B901B093BA011F910F91A5
:103410000C941B160F931F930091B7011091B801E4
:103420002091B9013091BA01DC01CB0180239123B5
:10343000A223B3238093B7019093B801A093B9015D
:10344000B093BA011F910F910C941B160F931F9309
:103450000091B7011091B8012091B9013091BA01E2
:10346000DC01CB0180279127A227B3278093B701E6
:103470009093B801A093B901B093BA011F910F9135
:103480000C941B161092B3011092B4011092B50166
:103490001092B6010C941B1641E050E060E070E021
:1034A00004C0440F551F661F771F8A95D2F74093BB
:1034B000B3015093B4016093B5017093B6010C94BD
:1034C0001B1641E050E060E070E004C0440F551F5F
:1034D000661F771F8A95D2F78091B3019091B4014E
:1034E000A091B501B091B601482B592B6A2B7B2BCB
:1034F0004093B3015093B4016093B5017093B6014A
:103500000C941B1641E050E060E070E004C0440FF2
:10351000551F661F771F8A95D2F740955095609585
:1035200070958091B3019091B401A091B501B091D3
:10353000B601482359236A237B234093B301509358
:10354000B4016093B5017093B6010C941B1641E071
:1035500050E060E070E004C0440F551F661F771F05
:103560008A95D2F78091B3019091B401A091B501F1
:10357000B091B601482759276A277B274093B301AA
:103580005093B4016093B5017093B6010C941B166F
:103590000F931F930091B3011091B4012091B501D5
:1035A0003091B601DC01CB01802B912BA22BB32BE8
:1035B0008093B3019093B401A093B501B093B60189
:1035C0001F910F910C941B160F931F930091B30141
:1035D0001091B4012091B5013091B601DC01CB010D
:1035E00080239123A223B3238093B3019093B4014A
:1035F000A093B501B093B6011F910F910C941B16C7
:103600000F931F930091B3011091B4012091B50164
:103610003091B601DC01CB0180279127A227B32787
:103620008093B3019093B401A093B501B093B60118
:103630001F910F910C941B160895CF92DF92EF9279
:10364000FF920F931F93CF93DF938C01C090B30130
:10365000D090B401E090B501F090B6018091B7012F
:103660009091B801A091B901B091BA01C82AD92AA4
:10367000EA2AFB2ACFE1D0E0D701C6010C2E04C014
:10368000B695A795979587950A94D2F780FF07C0BE
:10369000B8018C2F0E947B088130910531F421976D
:1036A00058F7B80180E00E947B08DF91CF911F910D
:1036B0000F91FF90EF90DF90CF90089590910C01C3
:1036C0009923F1F090910D019923D1F0982F9695BF
:1036D000969596959F3080F5E0910E01F0910F013F
:1036E000E90FF11D877021E030E0A90102C0440F0D
:1036F000551F8A95E2F7CA019181892B818308952C
:1037000020910E0130910F01F90132969FEF40E0B8
:103710005191851789F09F3F19F4511101C0942FE1
:103720004F5F4E30A9F79F3F39F0F901E90FF11DC6
:1037300097FDFA9582830895089590910C0199233D
:10374000F9F090910D019923D9F0982F96959695BF
:1037500096959F3028F5E0910E01F0910F01E90F49
:10376000F11D877021E030E0A90102C0440F551F10
:103770008A95E2F7CA018095918189238183089512
:1037800020910E0130910F01F9013296205F3F4FD9
:103790009081891301C010823196E217F307C1F7B7
:1037A000089581E090E0E0910E01F0910F01E80FA3
:1037B000F91F1082019680319105A9F70895909123
:1037C000CD01892B8093CD01089580959091CD01F5
:1037D00089238093CD0108951092CD010895909191
:1037E000CC01892B8093CC01089580959091CC01D8
:1037F00089238093CC0108951092CC010895809381
:10380000BB0108951092BB01089580910E01909123
:103810000F01FC0131969C01205F3F4F80E09191A8
:1038200091118F5FE217F307D1F70895E0910E0130
:10383000F0910F018091CD018083E0910E01F09114
:103840000F0190818091CC01892B80838091BB01F5
:10385000882361F0E0910E01F0910F019081892B96
:1038600080830E94051C81111092BB0180910E0182
:1038700090910F010C94D010CF92DF92EF92FF92B3
:103880006C01EE24FF24C114D104E104F10421F001
:10389000C701B60120E101C020E0C72ED82EE92ED5
:1038A000FF24C114D104E104F10419F0285FC70119
:1038B000B6016B017C0154E0F694E794D794C79469
:1038C0005A95D1F7C114D104E104F10419F02C5F29
:1038D000C701B6016B017C0142E0F694E794D794EE
:1038E000C7944A95D1F7C114D104E104F10419F049
:1038F0002E5FC701B601DC01CB01B695A795979560
:103900008795892B8A2B8B2B09F02F5F822FFF90B5
:10391000EF90DF90CF9008958091E601843011F10F
:1039200020E488E190E00FB6F894A89580936000B9
:103930000FBE2093600083B7817F846083BF83B70D
:10394000816083BF7894889583B78E7F83BF0FB6DD
:10395000F894A8958091600088618093600010922F
:1039600060000FBE089508950C94B31CCF930E947D
:10397000B41C0E949A060E94B31CC0E08C2F0E94C7
:103980009007811104C0CF5FCE30C1F701C081E044
:10399000CF9108950E942D160E94C4100C94BA096C
:1039A00082E084BD93E095BD9AEF97BD80936E0051
:1039B00008952FB7F8948091CF019091D001A091F4
:1039C000D101B091D2012FBF0895CF92DF92EF9233
:1039D000FF920F931F932FB7F8944091CF0150910E
:1039E000D0016091D1017091D2012FBF6A017B019A
:1039F000EE24FF248C0120E030E0C016D106E20660
:103A0000F30610F4415051099A01281B390BC901E2
:103A10001F910F91FF90EF90DF90CF9008951F922C
:103A20000F920FB60F9211248F939F93AF93BF9372
:103A30008091CF019091D001A091D101B091D2019C
:103A40000196A11DB11D8093CF019093D001A09349
:103A5000D101B093D201BF91AF919F918F910F90FF
:103A60000FBE0F901F9018950E94BC0DF8942FEF79
:103A700087EA91E6215080409040E1F700C00000C5
:103A800087E090EBDC018093EF019093F001A0932D
:103A9000F101B093F2019CE088E10FB6F894A8958B
:103AA000809360000FBE90936000FFCFEF92FF9273
:103AB0000F931F93CF93DF93D82FC0E08C2F0E94DA
:103AC000900700E010E0E82EF12CC701002E02C0A4
:103AD000959587950A94E2F780FD06C00F5F1F4F0A
:103AE0000630110591F709C0602F7C2F80E00E94FD
:103AF00058088D13F3CF81E004C0CF5FCE30F1F6CC
:103B000080E0DF91CF911F910F91FF90EF9008958A
:103B1000CF93C82F8CE20E94561D882321F08C2F52
:103B2000CF910C94561D80E0CF910895CF930E94C1
:103B3000DD1E811102C00E94C31EC5E6C15049F0BE
:103B40000E949A068FE39CE90197F1F700C00000FC
:103B5000F5CF89E20E94881D811113C18AE20E947B
:103B6000881D81110E94C31E85E00E94881D81115D
:103B70000E94341D0E94E81E8093CE0187E00E94BF
:103B8000881D8823A9F18BE10E94881D882351F0AC
:103B90008091CE0181FB222720F991E0922790FBB2
:103BA00081F90EC08EE00E94881D882361F080910B
:103BB000CE0182FB222720F991E0922790FB82F927
:103BC0008093CE0115C080E10E94881D9091CE01A6
:103BD000882341F093FB222720F981E0822780FB94
:103BE00093F904C0892F809580FB90F99093CE01C2
:103BF0008091CE010E94EC1E0E94FA1E8093E0018B
:103C000080EE0E94881D882341F08091E001982F6A
:103C1000909590FB80F98093E00189E30E94881DD4
:103C2000882359F08091E00181FB222720F991E05F
:103C3000922790FB81F98093E00182EE0E94881D1B
:103C4000882359F08091E00182FB222720F991E03E
:103C5000922790FB82F98093E00186EE0E94881DF6
:103C6000882359F08091E00183FB222720F991E01D
:103C7000922790FB83F98093E00183EE0E94881DD8
:103C8000882359F08091E00184FB222720F991E0FC
:103C9000922790FB84F98093E00185E30E94881DC0
:103CA000882359F08091E00185FB222720F991E0DB
:103CB000922790FB85F98093E00181E30E94881DA3
:103CC000882359F08091E00186FB222720F991E0BA
:103CD000922790FB86F98093E00181E10E94881D84
:103CE000882359F08091E00187FB222720F991E099
:103CF000922790FB87F98093E0018091E0010E9478
:103D0000FE1E8091E00187FB882780F980930D01DA
:103D100087E20E94881DC82F8EE10E94881D8111B4
:103D2000C2608FE10E94881D8111C46080E20E9400
:103D3000881D8111C86081E20E94881D8111C061C7
:103D400082E20E94881D8111C06283E20E94881D68
:103D50008111C06484E20E94881D882311F0C0682C
:103D600002C0CC2329F08C2F0E94F51E6C2F03C0BB
:103D70000E94F11E682F70E080E090E0CF910C94DB
:103D8000E419CF9108956DEE7EEF80E090E00E94FF
:103D9000372560E082E090E00E94292560E083E022
:103DA00090E00E94292560E084E090E00E942925AF
:103DB00060E085E090E00C94292580E090E00E948E
:103DC000232521E08D3E9E4F09F020E0822F0895AB
:103DD00082E090E00C941B25682F82E090E00C9428
:103DE000292583E090E00C941B25682F83E090E068
:103DF0000C94292584E090E00C941B25682F84E026
:103E000090E00C9429258091D50180FF0BC0609132
:103E1000130185E0689FB00111247595679575952C
:103E200067952BC081FF09C06091130185E0689FF1
:103E3000B00111247595679520C082FF07C060917D
:103E4000130185E0689FB001112417C09091D6013D
:103E50009923D1F060911201961788F720911301F0
:103E600085E0289F90011124929FA001939F500DFF
:103E7000112470E0CA010E94ED246038710540F4FD
:103E80006115710519F406C065E070E0862F08958C
:103E90008FE7089581E008958091D50180FF08C0E3
:103EA0006091110170E0759567957595679521C0D2
:103EB00081FF06C06091110170E07595679519C08A
:103EC00082FF04C06091110170E010C09091D60192
:103ED000992399F0609110019617A0F78091110134
:103EE000899FC001112470E00E94ED2460387105A3
:103EF00040F46115710519F406C061E070E0862F89
:103F000008958FE7089581E00895803F21F40E948D
:103F1000031F819504C0813F29F40E94031F8093F1
:103F2000D9010895823F21F40E94031F819504C0A6
:103F3000833F29F40E94031F8093D8010895893F8D
:103F400019F40E944C1F05C08A3F31F40E944C1F97
:103F500081958093DA0108958B3F21F40E944C1FD4
:103F6000819504C08C3F29F40E944C1F8093DB0193
:103F70000895843F21F48091D701816017C0853F67
:103F800021F48091D701826011C0863F21F4809195
:103F9000D70184600BC0873F21F48091D7018860EE
:103FA00005C0883F31F48091D70180618093D701AB
:103FB00008958D3F21F48091D50181600BC08E3F23
:103FC00021F48091D501826005C08F3F29F4809152
:103FD000D50184608093D5010895803F39F48091A4
:103FE000D90187FF6CC01092D90169C0813F29F4C3
:103FF0008091D9011816BCF362C09091D801823F1C
:1040000029F497FF5CC01092D80159C0833F19F47E
:104010001916CCF354C0893F41F48091DA01181687
:104020000CF04DC01092DA014AC08A3F29F4809109
:10403000DA0187FF44C0F6CF8B3F39F48091DB0172
:1040400087FF3DC01092DB013AC08C3F29F480917C
:10405000DB011816BCF333C0843F21F48091D701F3
:104060008E7F17C0853F21F48091D7018D7F11C0CD
:10407000863F21F48091D7018B7F0BC0873F21F4CD
:104080008091D701877F05C0883F31F48091D701A7
:104090008F7E8093D70113C08D3F21F48091D5018D
:1040A0008E7F0BC08E3F21F48091D5018D7F05C09E
:1040B0008F3F29F48091D5018B7F8093D50180912A
:1040C000D80181110EC08091D90181110AC080915F
:1040D000DA01811106C08091DB01811102C01092CA
:1040E000D601089587ED91E00E94DB100E94D91C53
:1040F0009093D4018093D30108951F93CF93DF93BE
:104100008091D3019091D4010E94E51CAC01909163
:10411000D601992321F02091140130E006C02091AE
:1041200015018AE0289F900111244217530708F4D3
:1041300085C08091D801C091D901D091DA01109148
:10414000DB01811107C0C11175C0D11173C01111FC
:1041500071C074C09F3F19F09F5F9093D6011816ED
:1041600024F40E94031F8093D8018091D80187FF17
:1041700005C00E94031F81958093D8011C1624F46A
:104180000E94031F8093D9018091D90187FF05C048
:104190000E94031F81958093D9016091D801662305
:1041A00031F1C091D901CC2311F1062E000C770B0F
:1041B000880B990B0E94F42323E333E343E35FE38B
:1041C0000E9458240E94BC236093D8016C2FCC0F0E
:1041D000770B880B990B0E94F42323E333E343E32B
:1041E0005FE30E9458240E94BC236093D9011D16EE
:1041F00024F40E944C1F8093DA018091DA0187FF3A
:1042000005C00E944C1F81958093DA01111624F499
:104210000E944C1F8093DB018091DB0187FF05C06A
:104220000E944C1F81958093DB01DF91CF911F91FC
:104230000C9472209F3F09F08FCFA0CFDF91CF91D8
:104240001F910895E7EDF1E085E0DF011D928A9569
:10425000E9F71092D6011092D5010895833081F1CB
:1042600028F4813059F08230D1F00895853009F476
:1042700049C0B8F1863009F456C0089580911501FF
:10428000262F30E0280F311D2F3F310524F4680F11
:104290006093150108958FEF809315010895809123
:1042A0001401262F30E0280F311D2F3F310524F453
:1042B000680F6093140108958FEF8093140108959F
:1042C00080911301262F30E0280F311D2F3F31053B
:1042D00024F4680F6093130108958FEF8093130106
:1042E000089580911201262F30E0280F311D2F3FB5
:1042F000310524F4680F6093120108958FEF8093C5
:104300001201089580911101262F30E0280F311DF0
:104310002F3F310524F4680F6093110108958FEF4A
:1043200080931101089580911001262F30E0280F0D
:10433000311D2F3F310524F4680F6093100108955B
:104340008FEF809310010895833011F128F48130AC
:1043500049F0823091F00895853081F120F1863066
:10436000C1F1089580911501681720F4861B809390
:104370001501089510921501089580911401681790
:1043800020F4861B8093140108951092140108955F
:1043900080911301681720F4861B80931301089500
:1043A00010921301089580911201681720F4861B62
:1043B00080931201089510921201089580911101C5
:1043C000681720F4861B8093110108951092110143
:1043D000089580911001681720F4861B80931001C6
:1043E00008951092100108950F931F938D3109F4D1
:1043F0006BC008F03FC08E3009F47DC0C0F4873038
:1044000009F46EC068F4863009F0AFC08091CE0127
:10441000817F8E7F8093CE0181E08093DD01A6C0F5
:10442000883009F458C08B3009F49BC09EC0863197
:1044300009F497C078F4803109F470C0813109F033
:1044400094C00E942D1690910D0181E089278093E0
:104450000D0187C0893109F484C08B3109F085C012
:104460008091CE0181FB222720F991E0922790FBD9
:1044700081F94AC0853309F45BC048F4873209F4F6
:1044800057C008F45AC0893209F452C06EC0833450
:1044900038F48A3308F067C0883309F462C065C015
:1044A000833409F445C0883409F05FC00E942D169A
:1044B0000FEF13ED20E3015010402040E1F700C062
:1044C00000000E94341D4DC00E9476230E94C4103B
:1044D0000E94BA0946C00E94E81E0E94FA1E41C00E
:1044E0009091CE01892F817090FF12C0917F9E7FA5
:1044F0009093CE013BC08091CE0182FB222720F910
:1045000091E0922790FB82F98093CE01992349F1A3
:104510008091CE0181608093CE0123C08091CE0135
:1045200083FB222720F991E0922790FB83F9ECCFBF
:1045300061E070E080E090E010C08D5141E050E01B
:1045400060E070E08A019B0104C0000F111F221F70
:10455000331F8A95D2F7C901B8010E94E4190E945D
:104560002D1681E003C08953E9CF80E01F910F91A0
:10457000089580E008950C94B922CF93C82F8091BC
:10458000DD01813079F018F08230E9F187C0E091E7
:104590000E01F0910F018081813169F0823209F0C2
:1045A0007FC009C0E0910E01F0910F01808181313F
:1045B00011F0823261F48C2F0E94BB22811104C061
:1045C0008C2F0E94F4211DC081E090E01AC08C2F36
:1045D0000E94B922811114C0C43179F048F4CB3063
:1045E00079F0C03109F060C082E08093DD0108C03D
:1045F000C93219F0C83321F057C01092DD0154C000
:1046000081E0817053C0C93289F118F5C43171F16C
:10461000A8F4C73009F046C08AE08093150194E100
:104620009093140193E0909313018093120188E01A
:104630008093110188E28093100134C0CE51C630BE
:1046400088F5EC2FF0E0E65DFE4F80818093DC0181
:1046500029C0CE34E9F020F4CB3421F56AE013C050
:10466000C13579F0C235F1F461E00DC08091DC0113
:10467000882319F01092DC0115C081E08093DD01E0
:1046800015C061E006C08091DC010E942E210AC0A5
:104690006AE08091DC010E94A42104C01092DD0137
:1046A00080E004C081E002C080E0ABCFCF910895EC
:1046B000E1E8F0E080818860808380818160808390
:1046C0008FB7F89493E09093890090ED90938800D1
:1046D0008FBF0895EFE6F0E08081826080830895C7
:1046E000EFE6F0E080818D7F80830895EFE6F0E0D3
:1046F000908182E08927808308951F920F920FB6E0
:104700000F9211242F933F934F935F936F937F9357
:104710008F939F93AF93BF93EF93FF938091DE01AD
:104720009091DF0101969093DF018093DE0181116A
:1047300003C082E00E94BA09E091DF01E695E695A8
:10474000F0E0E156F84FE4918091DE018E1303C052
:1047500080E00E94BA09FF91EF91BF91AF919F91C4
:104760008F917F916F915F914F913F912F910F901A
:104770000FBE0F901F9018950E94C3236894B1112B
:104780000C94522408950E94372488F09F5798F083
:10479000B92F9927B751B0F0E1F0660F771F881F46
:1047A000991F1AF0BA95C9F714C0B13091F00E9460
:1047B0005124B1E008950C945124672F782F882755
:1047C000B85F39F0B93FCCF3869577956795B39587
:1047D000D9F73EF490958095709561957F4F8F4FF6
:1047E0009F4F0895E89409C097FB3EF490958095FB
:1047F000709561957F4F8F4F9F4F9923A9F0F92FA7
:1048000096E9BB279395F695879577956795B79524
:10481000F111F8CFFAF4BB0F11F460FF1BC06F5F0A
:104820007F4F8F4F9F4F16C0882311F096E911C01C
:10483000772321F09EE8872F762F05C0662371F03D
:1048400096E8862F70E060E02AF09A95660F771F51
:10485000881FDAF7880F9695879597F9089557FD81
:104860009058440F551F59F05F3F71F04795880FDE
:1048700097FB991F61F09F3F79F087950895121675
:1048800013061406551FF2CF4695F1DF08C0161621
:1048900017061806991FF1CF8695710561050894D2
:1048A0000895E894BB2766277727CB0197F90895E9
:1048B0000E946B240C94DC240E94CE2438F00E94C9
:1048C000D52420F0952311F00C94C5240C94CB240E
:1048D00011240C9452240E942F2470F3959FC1F34D
:1048E000950F50E0551F629FF001729FBB27F00D9E
:1048F000B11D639FAA27F00DB11DAA1F649F6627F3
:10490000B00DA11D661F829F2227B00DA11D621F41
:10491000739FB00DA11D621F839FA00D611D221FFB
:10492000749F3327A00D611D231F849F600D211DDF
:10493000822F762F6A2F11249F5750409AF0F1F062
:1049400088234AF0EE0FFF1FBB1F661F771F881FCB
:1049500091505040A9F79E3F510580F00C94C5241A
:104960000C9452245F3FE4F3983ED4F386957795F8
:104970006795B795F795E7959F5FC1F7FE2B880F71
:10498000911D9695879597F9089597F99F6780E807
:1049900070E060E008959FEF80EC089500240A9491
:1049A0001616170618060906089500240A9412160A
:1049B0001306140605060895092E0394000C11F43D
:1049C000882352F0BB0F40F4BF2B11F460FF04C0EA
:1049D0006F5F7F4F8F4F9F4F089597FB072E16F401
:1049E000009407D077FD09D00E94072507FC05D069
:1049F0003EF4909581959F4F0895709561957F4FF6
:104A00000895EE0FFF1F0590F491E02D0994AA1B65
:104A1000BB1B51E107C0AA1FBB1FA617B70710F0A9
:104A2000A61BB70B881F991F5A95A9F780959095DB
:104A3000BC01CD010895F999FECF92BD81BDF89AD0
:104A4000992780B50895A8E1B0E042E050E00C94C9
:104A50003E25262FF999FECF1FBA92BD81BD20BDFC
:104A60000FB6F894FA9AF99A0FBE019608950E942B
:104A70002925272F0C942A25DC01CB01FC01F9996B
:104A8000FECF06C0F2BDE1BDF89A319600B40D929A
:0C4A900041505040B8F70895F894FFCF53
:104A9C002002BB094B0A260AF209BE090101BC011E
:104AAC0028080A03140A3F4D363960071307DD0640
:104ABC00A4063706500669068206010203040506A1
:044ACC0007080900CE
:00000001FF
